:020000040000FA
:10000000831603138101E0298B138B1B04289600B0
:10001000030E970083010A0898008A0183130408DD
:1000200099009308031D1728051A3328362813084A
:10003000083C031C2328051E9413051A9417031962
:100040003628940C36281308093C031C2828362827
:10005000051E33281017831603130610831203138B
:1000600006100B123428940193013728930A8B1041
:100070001908840018088A00170E8300960E160EC1
:10008000090014089500F03C031D492810141011B4
:100090002829101CE32810101408123C03195328B7
:1000A0001408593C031990101408583C031D5E288D
:1000B000901D5C2890112829901528291408113CBE
:1000C000031D6428101236291408143C031D282926
:1000D00090123629820700343934003435343334F1
:1000E0003134323432340034303438343634343409
:1000F00009347E3400340034322930290034342964
:10010000713431340034003400347A34733461345F
:1001100077343234003400346334783464346534F2
:100120003434333400340034203476346634743458
:1001300072343534003400346E34623468346734D9
:10014000793436340034003400346D346A34753414
:1001500037343834003400342C346B3469346F3421
:1001600030343934003400342E343F346C343B3472
:1001700070342D34003400340034273400345B34C0
:100180002B34003400340034302924295D34003409
:100190007C340034003400343C3430342E34323477
:1001A0003534363438340034003431342B3433347D
:1001B0002D342A34393400340834003400343134D6
:1001C000373434343734101DF12814084A3C031DE9
:1001D000EC282F309400212914085A3C0318F128E8
:1001E00028291408613C031807290E3094021408CA
:1001F000613C031CFE281930940707291408773C3A
:10020000031807291408D23C0319101528290030B7
:100210008A0014086A2094009408031928291408F5
:10022000603C0318372914087A3C031C372914084A
:1002300090191D29901C21291F2990182129E03E81
:1002400094001408A72128290D30A7210A3008009E
:100250008316031306148312031310130B160800DE
:100260009014003410160034901600342829901C85
:10027000212914080D3C031821291508613C031C91
:10028000212915083C3C031848293D309502512985
:100290001508243C03184F292330950251290430B6
:1002A000950701308A0015085721940021298207FB
:1002B00026342A34243423343C34003400340034CB
:1002C00029342834003425343E342F3400343A3471
:1002D00000345F3460345E340034223400347B34C4
:1002E0003D34003421340034003400347D34003493
:0A02F0005C340034403400343E3426
:100320008C00810183160313C030810508008C0006
:10033000810183160313C0308105013081048312CB
:1003400003130B110B1DA2298C0BA129080091008E
:10035000051008308C00B82111180514111C051067
:10036000910CB8218C0BAC290514B821B8210800D8
:100370001D308D00BE2908308D00BE298D0BBE2991
:060380000800920137287D
:1003C0000510831203130514831603130614051670
:1003D0000113831203130B1693019001F8308B0560
:1003E0008B172A308E0002308A000E082A3C102219
:0C03F000A7218E0BF329101B4120FB29D4
:10042000820750344934433420343134363446342E
:100430003834343420344134543420344B3465342B
:10044000793462346F346134723464342034443427
:10045000653463346F346434653472342034633407
:100460006F346E346E34653463347434653464349C
:060470000D340A340A34C9
:02400E00F13F80
:00000001FF
